:100000004529A01123080319A0150530A2002730A7
:10001000A900103017200330A900E8301720A901EB
:1000200064301720A9010A3017202C081E28A800C8
:100030002D08A5002C08A400DB202408A400A2039E
:100040000319A011230803192828220203182F28B6
:100050002408031DA011A0192F28303E35280800C0
:100060000C1E30289900031440292119302808005B
:1000700083169B0083161C141A089B0A4029A901A9
:10008000A800FF30A807031CA907031C4029033060
:10009000A500E5304D204128A501F63EA400A509A4
:1000A000031C5828FE300000A40703185328A40797
:1000B0000000A50F5228000024185E28241860288C
:1000C000080027082F068039B100A71F7228A4094D
:1000D000A509A609A709A40A0319A50A0319A60ACE
:1000E0000319A70AAF1F7F28AC09AD09AE09AF09F4
:1000F000AC0A0319AD0A0319AE0A0319AF0AA80125
:10010000A901AA01AB01B601B701B801B9012F08D5
:100110002E042D042C040319BD282030B000031038
:10012000A40DA50DA60DA70DB60DB70DB80DB90DF3
:100130002F083902031DA6282E083802031DA62801
:100140002D083702031DA6282C083602031CB728E9
:100150002C08B6022D08031C2D0FB7022E08031C15
:100160002E0FB8022F08031C2F0FB9020314A80D7D
:10017000A90DAA0DAB0DB00B8F28B11FCA28A80975
:10018000A909AA09AB09A80A0319A90A0319AA0A05
:100190000319AB0A3608AC003708AD003808AE00CA
:1001A0003908AF002808A4002908A5002A08A600DD
:1001B0002B08A7004029AD01AC011030B000250D7F
:1001C000AC0DAD0D2808AC022908031C290FAD02A7
:1001D0000318F1282808AC0729080318290FAD07D0
:1001E0000310A40DA50DB00BDF28240840292030F2
:1001F000B000B601B701B801B9010310241C0E29E3
:100200002C08B6072D0803182D0FB7072E08031862
:100210002E0FB8072F0803182F0FB907B90CB80C09
:10022000B70CB60CA70CA60CA50CA40CB00BFD28A3
:1002300008001030B300A501A401B10CB00C031CE0
:1002400027292808A40729080318290FA507A50CA2
:10025000A40CAD0CAC0CB30B1D292C084029A40038
:10026000A71B342124084029A409A509A609A70928
:10027000A40A0319A50A0319A60A0319A70A080064
:100280008313831203130000080083160F309900B4
:1002900020309800831280309800A0010130900037
:1002A00097014A3083168600FD308500073083129F
:1002B0009F008A11492A8E018F010530970083160D
:1002C0000C1183120C1183160C1583128A110C1950
:1002D0006B298A0165291508D0001608D100043061
:1002E00097000C118A110C1977298A0172291508B7
:1002F000D2001608D30050085202D6005108031C41
:10030000013E5302D700053097000C118A110C19D9
:100310008B298A0186291508D4001608D5000C11EE
:1003200050085402D8005108031C013E5502D90060
:1003300083160C1183129701570859028A11031C66
:10034000E1298A11031DA929560858028A11031CA4
:10035000E1295B08D602031CD7035A08DC001030E1
:10036000DD00A701A6015D08A5005C08A400AF019F
:10037000AE015708AD005608AC008A01F7202708E7
:10038000CE002608CD002508CC002408CB004E085E
:10039000A7004D08A6004C08A5004B08A400AF011B
:1003A000AE015908AD005808AC008A016120270849
:1003B000CE002608CD002508CC002408CB008A11E9
:1003C000E529CE01CD01CC01CB018A11CE1BFF293D
:1003D0004D084E048A11031DFA2910304C028A116F
:1003E000031CFF298A11031DFA2901304B028A11CF
:1003F000031CFF29CE01CD011030CC00CB018A11A6
:10040000CE1F062ACE01CD01CC01CB0108003B084E
:10041000B1003A08B000A9012D30A8008A011921C5
:10042000C5002D08C6004608C300C4010310C30C54
:100430004508C70001304605C8004808B100470814
:10044000B000A9010A30A8008A011921C7002D08AF
:10045000C8004808C900CA010310C90C4708C500F4
:1004600001304805C600013046028A11031C482AA3
:100470004908093A4A048A11031D452AC30A031987
:10048000C40ACA01C9018A11482AC90A0319CA0A39
:10049000080064308A013F200130CF0000308A011B
:1004A0003820C20001308A013820DA0002308A0187
:1004B0003820DB008A015B214C08BB004B08BA00E6
:1004C0008A1186188C2A86163B08AD003A08AC00C3
:1004D000AE01AF01003EBC00F030BD002D08031896
:1004E0002D0FBD07FF30BE002E0803182E0FBE07CC
:1004F000FF30BF002F0803182F0FBF073F08A700CA
:100500003E08A6003D08A5003C088A012F21BA003C
:100510002508BB008A118D2A86128A110519A42A82
:1005200006160830BB0710303B028A11031CA22AB2
:100530008A11031DA02A01303A028A11031CA22A43
:100540001030BB028A11A52A06128A11061B762BCF
:100550008A118519292B8A010722C2088A11031DD5
:10056000EA2A41308A0130205A308A01302049304D
:100570008A0130204D308A01302055308A013020E8
:1005800054308A01302048308A01302020308A01DE
:1005900030203D308A01302020308A013020043064
:1005A000A100A3014408AD004308AC008A0101206A
:1005B0002E308A013020A3014A08AD004908AC0062
:1005C0008A01012020308A0130200D308A0130203C
:1005D0008A11272B45308A0130204C308A01302087
:1005E00045308A01302056308A01302041308A015E
:1005F000302054308A01302049308A0130204F3079
:100600008A0130204E308A01302020308A0130208B
:100610003D308A01302020308A0130200430A10092
:10062000A3014408AD004308AC008A0101202E302C
:100630008A013020A3014A08AD004908AC008A01B4
:10064000012020308A0130200D308A0130208A11AB
:10065000712BC2088A11031D512B0130CF0041308C
:100660003A07B4003B080318013EB5004F083407B1
:10067000C00035080318013EC10041308A01302016
:100680003A088A0130203B088A0130204F088A014D
:10069000302040088A01302041088A0130208A1128
:1006A000712B45303A07B4003B080318013EB500F2
:1006B0004F083407C00035080318013EC10045301B
:1006C0008A0130203A088A0130203B088A01302014
:1006D0004F088A01302040088A01302041088A01F1
:1006E00030208A11061B762B8A01712B8A015A2A27
:0606F00063008A01782B73
:02400E00223F4F
:0642000000000D000B00A0
:00000001FF
